:020000040000FA
:0400000050EF01F0CC
:08000800056ED8CF06F0E0CF31
:1000100007F00001E9CF0DF0EACF08F0E1CF09F0D9
:10002000E2CF0AF0D9CF0BF0DACF0CF0F3CF14F017
:10003000F4CF15F0FACF16F000C00FF001C010F0A9
:1000400002C011F003C012F004C013F09DA22CEF07
:1000500000F09EB283EF00F00FC000F010C001F07E
:1000600011C002F012C003F013C004F00DC0E9FF8C
:1000700008C0EAFF09C0E1FF0AC0E2FF0BC0D9FFD8
:100080000CC0DAFF14C0F3FF15C0F4FF16C0FAFF6E
:10009000055007C0E0FF06C0D8FF1000F2CF0EF0F9
:1000A000F29EF76AB60FF66E000EF7220900F550C1
:1000B0000EBEF28E120001020408102040800000E3
:1000C000016A026A006A036A405002E13F5018E088
:1000D000100E416ED8903D363E3600360336405005
:1000E000035C02E13F50005C07E33F50005ED8A094
:1000F00003064050035ED88001360236412EEAD70F
:1001000000008EEF00F0182AD8B4192A19C03EF06A
:1001100018C03DF0406A640E3F6ED2D700C018F0A0
:1001200003C019F0195203E11B50185C03E38A80E5
:10013000939002D08A909390195203E11C50185C5E
:1001400003E38A86939602D08A969396195203E126
:100150001D50185C03E38A8C939C02D08A9C939C6C
:100160009E922CEF00F0180E386E396A3850395CC8
:1001700012E28A9293928A8A939A020E006E002E5D
:10018000FED700008A9A939A020E006E002EFED7C8
:100190000000392AEBD7000C8A889398020E006E73
:1001A000002EFED700008A989398000CFF0E926EE6
:1001B00080CF38F0C2B2FED7C3CF39F0C4CF3AF007
:1001C00038A204D01AB402D01A841A8A1AA400D011
:1001D00038A404D01AB602D01A861A8A1AA600D0F9
:1001E00038A604D01AB802D01A881A8A1AA800D0E1
:1001F00038A803D01AB201D01A821AA204D03AC089
:100200001FF039C01EF01E0E39241E6E000E3A205B
:100210001F6E385205E11A941A961A981A921A9A71
:10022000C282000C3B6A3B50070826E338A003D08B
:100230008A82939202D08A92939239A003D08A84C0
:10024000939402D08A9493943AA003D08A8E939E7A
:1002500002D08A9E939E8A8A939A020E006E002E86
:10026000FED700008A9A939AD8903832D8903932C3
:10027000D8903A323B2AD7D7000C3B6A3A6A3B50B7
:10028000395C0DE303E138503A5C09E21A0E006E66
:10029000002EFED700003A2AD8B43B2AF0D7000C33
:1002A000F86AD09E0D8EEA6AE96AC29CC29EC1506D
:1002B000800B7F09C16E186A196A1A921A941A96ED
:1002C0001A981A9A3C0E1B6E280E1C6E1D6E320E6A
:1002D0001E6E1F6A216A226A236A246A256A266AB8
:1002E000276A286A296A2A6A2B6A2C6A2D6A2F6A69
:1002F000306A316A326A336A376AF19EC29CC29EA2
:10030000C150800B7E09C16EC050C00B0709C06E82
:10031000C08EC280000E016EC250E30B0110C26E8F
:10032000D190800ED56ECD6A080E0509CA6E180EE2
:10033000CB6EB150480BB16E9D82C00EF2128A9204
:1003400093928A9493948A9E939E0DDF25DF8A90E0
:1003500093908A9C939C8A96939605DF2E6A2E50E2
:1003600017085CE32E302D6E2D322D321F0E2D1608
:10037000216A226A236A020ED8802D54036A210F53
:10038000E96E000E0320EA6E2E50070B036AF2CFCF
:100390003CF0F29E83DE3CBEF28EEF6E07DF206AF9
:1003A0002050020830E332A00AD0036A2050210F07
:1003B000E96E000E0320EA6EEFCF34F001D0346A0C
:1003C00032A20AD0036A2050210FE96E000E0320EA
:1003D000EA6EEFCF35F001D0356A32A40AD0036A55
:1003E0002050210FE96E000E0320EA6EEFCF36F0A9
:1003F00001D0366A34C038F035C039F036C03AF032
:1004000011DF202ACDD7C8DE1AAA01D02E061FC0C0
:1004100039F01EC038F031DF2E2AA1D7160E2E6E0D
:100420002E525CE02E302D6E2D322D321F0E2D16E9
:10043000216A226A236A020ED8802D54036A210F92
:10044000E96E000E0320EA6E2E50070B036AF2CF0E
:100450003CF0F29E23DE3CBEF28EEF6EA7DE206AF9
:100460002050020830E332A00AD0036A2050210F46
:10047000E96E000E0320EA6EEFCF34F001D0346A4B
:1004800032A20AD0036A2050210FE96E000E032029
:10049000EA6EEFCF35F001D0356A32A40AD0036A94
:1004A0002050210FE96E000E0320EA6EEFCF36F0E8
:1004B00001D0366A34C038F035C039F036C03AF071
:1004C000B1DE202ACDD768DE1AAA01D02E061FC0C1
:1004D00039F01EC038F0D1DE2E06A2D7010E32242C
:1004E000070B326E325202E1010E326E36D7030034
:020000040030CA
:0E00000000060E0E0080810003C003E00340E6
:00000001FF
